:100000000C945B000C9481000C9481000C94810092
:100010000C9481000C9481000C9481000C9481005C
:100020000C9481000C9481000C9481000C9481004C
:100030000C9481000C9481000C9481000C9481003C
:100040000C94A8020C9481000C9482040C948100FE
:100050000C9481000C9481000C9481000C9481001C
:100060000C9481000C948100A7020000000700029C
:10007000010000030406000000000000000001026F
:100080000408102040800102040810200102040826
:100090001020040404040404040402020202020204
:1000A0000303030303030000232629000025282B54
:1000B000000024272A0011241FBECFEFD4E0DEBFAA
:1000C000CDBF11E0A0E0B1E0ECEFFBE002C0059095
:1000D0000D92A231B107D9F711E0A2E1B1E001C060
:1000E0001D92A93AB107E1F710E0CAE6D0E004C0DA
:1000F0002297FE010E94FA05C836D107C9F70C9471
:1001000021010C94000008950F931F93CF93DF9368
:10011000EC018C01000F111FF801E45EFE4F11820B
:100120001082095F1E4F61E0F80180810E94560332
:1001300060E0F80180810E94BD0382E090E00E94AF
:10014000070361E0F80180810E94BD0385E090E033
:100150000E94070360E0F80180810E94BD0360E017
:10016000F80180810E945603F80105C0FE01EE0FE0
:10017000FF1FE95FFE4F80810E94740390931B0173
:1001800080931A0180911A0190911B01892B71F3C0
:1001900015C08E01000F111FF801E95FFE4F80812D
:1001A0000E94740390931B0180931A01045E1E4FFA
:1001B000F8018081918101969183808380911A0159
:1001C00090911B01019729F3DF91CF911F910F911E
:1001D00008950F931F9300E211E06BE071E0C801F6
:1001E0000E94EC0160911C0170911D01C8010E94E8
:1001F00093026EE071E0C8010E940C021F910F9102
:10020000089540E051EE60E070E080E291E00E94ED
:10021000D90161E0809107010E94560360E080915E
:1002200007010E94BD03089580E090E00E948400D1
:100230000E94E90064E170E080E090E00E94E50245
:100240000895CFEFD4E0DEBFCDBF0E9414030E941B
:1002500001010E941401FDCFA2C080E291E00E9442
:10026000E201809306019927AA27BB2720E030E00E
:10027000AC01BD0180E291E00E947802409106014C
:10028000842F81548A31A8F4409304011092030111
:1002900010920201E2E1F1E087E090E01192119208
:1002A000019797FFFBCF8FEF9FEF90930301809310
:1002B00002014D3231F48FEF9FEF90930101809353
:1002C0000001842F80538A30C8F4E0910201F0913C
:1002D0000301EE0FFF1FEE5EFE4F808191819C01B6
:1002E000A3E0220F331FAA95E1F7880F991F820F11
:1002F000931F840F911DC09791838083403259F5DD
:1003000040910201509103016FEF4F3F5607E1F01A
:10031000DCF0FA01EE0FFF1FEE5EFE4F20910001B0
:100320003091010180819181BC01269FC001279FEE
:10033000900D369F900D11249183808381E090E091
:1003400090930101809300014F5F5F4F5093030131
:100350004093020124C0413221F04A3011F04D3067
:10036000F1F4E0910201F0910301EE0FFF1FEE5E48
:10037000FE4F209100013091010180819181AC01FB
:10038000249FC001259F900D349F900D11249183CF
:10039000808381E090E0909301018093000180E2EE
:1003A00091E00E94DE01882309F057CF0895089557
:1003B0000895CB01BA010E94080408950E944904DF
:1003C000992708950E945A0408950E947904089577
:1003D000862F0E94C0040895CB010E94C70408958F
:1003E000862F0E94C00408950F931F938C016DE027
:1003F0000E94E8016AE0C8010E94E8011F910F9184
:1004000008950F931F938C010E94E801C8010E9478
:10041000F4011F910F9108950F931F938C010E9477
:10042000EC01C8010E94F4011F910F9108950F93F0
:100430001F938C010E94F001C8010E94F4011F91DA
:100440000F910895CB01BA013327442755270E9405
:10045000D40408952AE00E94220208950F931F9366
:100460008C010E942A02C8010E94F4011F910F9181
:100470000895AB01662777270E942A0208950F93FB
:100480001F938C010E943902C8010E94F4011F9140
:100490000F910895EF92FF920F931F93CF93DF93E5
:1004A000EC017A018B0177FF0BC06DE20E94E8013D
:1004B00010950095F094E094E11CF11C011D111DB4
:1004C0002AE0B801A701CE010E942202DF91CF915C
:1004D0001F910F91FF90EF9008950F931F938C0140
:1004E0000E944A02C8010E94F4011F910F910895D1
:1004F0002115310521F4642F0E94E80108952A3066
:10050000310519F40E944A0208950E9422020895BA
:100510000F931F938C010E947802C8010E94F4017E
:100520001F910F910895AB01662757FD6095762FB7
:100530000E944A0208950F931F938C010E94930218
:10054000C8010E94F4011F910F9108950895089524
:100550001F920F920FB60F9211248F939F93AF9318
:10056000BF938091250190912601A0912701B09120
:1005700028010196A11DB11D8093250190932601AC
:10058000A0932701B0932801BF91AF919F918F91C4
:100590000F900FBE0F901F901895609125017091DC
:1005A0002601809127019091280127E0660F771F8F
:1005B000881F991F2A95D1F72DE730E040E050E0E1
:1005C0000E94A705CA01B9010895AF92BF92CF92C8
:1005D000DF92EF92FF920F931F935B016C010E94D9
:1005E000CD027B018C010E94CD026E197F09800B28
:1005F000910B6A157B058C059D05A8F31F910F9142
:10060000FF90EF90DF90CF90BF90AF90089501974B
:1006100051F0880F991F880F991F02972FB7F894F0
:100620000197F1F72FBF0895789410922501109249
:100630002601109227011092280184B5826084BDA2
:1006400084B5816084BD85B5826085BD85B58160D6
:1006500085BDEEE6F0E0808181608083E1E8F0E036
:10066000808182608083808181608083E0E8F0E027
:10067000808181608083E1EBF0E080818460808311
:10068000E0EBF0E0808181608083EAE7F0E0808148
:1006900084608083808182608083808181608083A8
:1006A0008081806880831092C1000895282F3327AD
:1006B000C90182589F4FFC0194912E563F4FF9017A
:1006C0008491882381F0E82FFF27E055FF4FE491C4
:1006D000FF27662329F480819095892380830895DC
:1006E0008081892B80830895482F5527CA01865918
:1006F0009F4FFC012491CA0182589F4FFC019491A5
:100700004E565F4FFA0134913323A1F1222331F188
:10071000233021F4809180008F7705C0243031F49C
:10072000809180008F7D8093800018C0213019F463
:1007300084B58F7704C0223021F484B58F7D84BDC9
:100740000DC0263021F48091B0008F7705C027308E
:1007500029F48091B0008F7D8093B000E32FFF27B4
:10076000EA55FF4FE491FF278081892319F081E04A
:1007700090E0089580E090E00895482F5527CA0141
:1007800086599F4FFC012491CA0182589F4FFC015A
:1007900094914E565F4FFA0134913323C1F12223D5
:1007A00031F1233021F4809180008F7705C024300F
:1007B00031F4809180008F7D8093800018C02130BB
:1007C00019F484B58F7704C0223021F484B58F7D6D
:1007D00084BD0DC0263021F48091B0008F7705C014
:1007E000273029F48091B0008F7D8093B000E32FF3
:1007F000FF27E555FF4FE491FF27662329F4808109
:1008000090958923808308958081892B8083089522
:10081000EF92FF920F931F937B018C0122E030E057
:1008200040E050E00E94C905205C3D4B404F5F4FC7
:10083000CA01B901A80197010E94C90521503040A1
:1008400040405040BB2757FDBA95A52F942F832FCA
:100850002F5F3F4F4F4F5F4F8093C5002150209334
:10086000C400E1ECF0E08081806180838081886059
:1008700080838081806880831F910F91FF90EF902B
:100880000895982F8091C00085FFFCCF9093C600FB
:1008900008958091230190912401209121013091AC
:1008A0002201821B930B80589F4F60E870E00E94EA
:1008B00094050895409121015091220180912301D6
:1008C000909124018417950719F48FEF9FEF0895F5
:1008D000FA01E75DFE4F2081CA01019660E870E0F1
:1008E0000E9494059093220180932101822F9927E1
:1008F0000895809121019091220190932401809389
:10090000230108951F920F920FB60F9211242F9377
:100910003F934F935F936F937F938F939F93AF9387
:10092000BF93EF93FF934091C600E0912301F091B4
:100930002401CF01019660E870E00E9494059C01BB
:1009400080912101909122012817390739F0E75D44
:10095000FE4F40833093240120932301FF91EF91B8
:10096000BF91AF919F918F917F916F915F914F91C7
:100970003F912F910F900FBE0F901F9018950895E3
:100980000E94410408958AE00E94C0040895CF9314
:10099000DF93EC0103C021960E94C0048881882364
:1009A000D1F7DF91CF9108952F923F924F925F92AE
:1009B0006F927F928F929F92AF92BF92CF92DF926F
:1009C000EF92FF920F931F93CF93DF93CDB7DEB7D4
:1009D000A0970FB6F894DEBF0FBECDBF6B017C01B0
:1009E00019012A01611571058105910521F480E342
:1009F0000E94C0044BC06624772443015E01089422
:100A0000A11CB11C8501060D171DC701B601A2016D
:100A100091010E94A705F80160830894611C711C74
:100A2000811C911CC701B601A20191010E94A7057A
:100A300069017A01211531054105510519F7730145
:100A40000894E108F108EA0CFB1CAA24BB24650108
:100A500011C0F70180818A3010F4805D01C0895C8B
:100A60000E94C0040894A108B108C108D1080894E4
:100A7000E108F10888279927DC0186199709A80958
:100A8000B909A816B906CA06DB0619F7A0960FB66B
:100A9000F894DEBF0FBECDBFDF91CF911F910F91B4
:100AA000FF90EF90DF90CF90BF90AF909F908F908E
:100AB0007F906F905F904F903F902F900895EF92AE
:100AC000FF920F931F937B018C0197FF0BC08DE268
:100AD0000E94C00410950095F094E094E11CF11C74
:100AE000011D111D2AE030E040E050E0C801B701CF
:100AF0000E94D4041F910F91FF90EF90089520E180
:100B000030E040E050E00E94D404089528E030E056
:100B100040E050E00E94D404089522E030E040E03C
:100B200050E00E94D404089597FB092E07260AD0AE
:100B300077FD04D049D006D000201AF47095619555
:100B40007F4F0895F6F7909581959F4F0895A1E204
:100B50001A2EAA1BBB1BFD010DC0AA1FBB1FEE1F37
:100B6000FF1FA217B307E407F50720F0A21BB30B82
:100B7000E40BF50B661F771F881F991F1A9469F7FE
:100B800060957095809590959B01AC01BD01CF015A
:100B9000089597FB092E05260ED057FD04D0D7DF08
:100BA0000AD0001C38F450954095309521953F4F60
:100BB0004F4F5F4F0895F6F790958095709561952A
:100BC0007F4F8F4F9F4F0895AA1BBB1B51E107C05A
:100BD000AA1FBB1FA617B70710F0A61BB70B881FCD
:100BE000991F5A95A9F780959095BC01CD0108955C
:0C0BF000EE0FFF1F0590F491E02D09941A
:100BFC000100FFFF40404008001900442000202164
:020C0C000000E6
:00000001FF
